:10000000789D001001030000090300000B030000AD
:100010000D0300000F030000110300004650FFEF26
:1000200000000000000000000000000013030000BA
:100030001503000000000000170300007903000012
:100040001B030000250300001B0300001B0300002E
:100050001B0300001B0300001B0300001B03000028
:100060001B0300001B0300001B0300001B03000018
:100070001B030000000000001B0300001B03000026
:100080001B0300001B0300001B0300001B030000F8
:100090001B0300001B0300001B0300001B030000E8
:1000A000EB2200001B0300001B0300001B030000E9
:1000B0001B0300001B0300001B0300001B030000C8
:1000C0001B0300001B0300001B0300001B030000B8
:1000D0001B0300001B0300001B0300001B030000A8
:1000E0001B030000DFF80CD004F07EFB0048004743
:1000F000710A0000789D0010D0F800D0D0F804F00C
:1001000070B50023084D0AE0CE5C04885B1C86EACB
:1001100014269BB235F8166086EA04240480521E29
:1001200092B2F1D270BD00003C4A000030B4554C90
:10013000534A0323C4F8B031136843F48033136087
:10014000514A30BC104710B572B633244F4B10C320
:1001500007C34F484FF47A710068B0FBF1F01860A4
:10016000191D4A48FFF7E2FF62B610BD474A322325
:100170001360C2E9010146484FF47A710068B0FB90
:10018000F1F0D06002F114011046CFE73F4A34236A
:100190001360C2E901013E484FF47A710068B0FB78
:1001A000F1F0D06002F114011046BFE710B572B64D
:1001B0000624384951F82420824212D93549783929
:1001C00051F82410814207D121460846FFF7CEFF9F
:1001D00021460846FFF7DAFF21460846FFF7C6FF2B
:1001E00002E0641C1D2CE5D962B610BD2DE9F0417A
:1001F000294C236803B92060244D0020283563680A
:1002000003E00F5C1E18401CAF559042F9D39818BC
:100210004FF480766060B04213D12068FFF7C6FFCC
:100220001A4D1435286800B1FEE7184932462831C6
:100230002068FFF788FF286800B1FEE700206060B3
:1002400020600020BDE8F08172B61449144A0140D4
:100250001160FFF751BF46F2044000210088A0F56D
:100260001942993A0AD04FF4C0404FF4002208C80E
:1002700090421944FBD309B1002070470120704718
:1002800088C10F4000C00F40F11FFF1F0C1C001061
:10029000DC000010F44D0000C400001080FFFF1FC0
:1002A00008ED00E0EFF3108010F0010F72B64FF090
:1002B00080404FF0000202704FF0AA0202724FF02D
:1002C000550303724FF0FF0444604FF003040470C1
:1002D0000272037200D162B6FEE710B50B46044607
:1002E0001146184604F06CFAC4E9000110BD02E0A2
:1002F00008C8121F08C1002AFAD17047FFFFFFFF8C
:100300000648804706480047FEE7FEE7FEE7FEE7AF
:10031000FEE7FEE7FEE7FEE7FEE7FEE75F1600000A
:10032000E500000010B54FF040210120086001F009
:10033000B0FB10BD10B54FF0E0241A4860611F21DA
:10034000601700F01EF80020A0610720206110BD9A
:10035000154810B5022141600021016741611D224D
:10036000C260C16301214160FFF7E4FF0221C81EA2
:1003700000F007F8002010BD0C480168491C01601E
:100380007047C906090E002806DA00F00F0000F1D8
:10039000E02080F8141D704700F1E02080F8001480
:1003A00070470000BFD4010000000940EC000010BD
:1003B00040EA01039B0703D009E008C9121F08C0E7
:1003C000042AFAD203E011F8013B00F8013B521E67
:1003D000F9D27047D2B201E000F8012B491EFBD2DE
:1003E00070470022F6E710B513460A460446194640
:1003F000FFF7F0FF204610BD70470000000000002E
:10040000000000004D0B0000FFB5ACA60446E1CE95
:100410008DE8E100022902DA002004B0F0BD601886
:10042000002100F8011D6946B3FBF2F502FB15350A
:10043000B3FBF2F34D5D00F8015DA042F4D8ECE7A8
:1004400010B504F0FDF804F0E7F8A0494FF40052AD
:10045000C1E90020A0F5F420886010BD70B5034606
:1004600008468D189949002449688D4200D9881A98
:10047000194604F034F9204670BDF8B51446934E81
:100480000A460B19716800258B4200D90A1B0346E6
:100490000094306804F04EF92846F8BD10B50B46BC
:1004A00001460024184604F0EEF8204610BD2DE960
:1004B000FC410746002090460E46ADF80000044679
:1004C0000EE0351B402D00D9402539192A468048B9
:1004D000FFF7E4FFAAB27E496846FFF711FE2C44FD
:1004E000B442EED33919424601A8FFF7D7FFBDF851
:1004F0000000BDF80410884202D10120BDE8FC8153
:100500000020FBE70021425C12B9491C1829FAD3EC
:10051000182901D000207047012070472DE9F041D3
:100520006A4C00270C3488B0A770E770DFF8A4810C
:100530004FF40056277101251922314601A8FFF713
:10054000ADFF022216213046FFF7B1FF00287DD013
:10055000DDF81210022206F11900FFF7A8FF0028AB
:1005600074D09DF8040006282AD2DFE800F02A03A0
:10057000032A2A1CD8F87410DDF80E30491C8B426F
:100580001ED2D8F87420DDF80E30D21ADDF8123001
:10059000521C9A4214D3DDF80E20DDF812301A44B2
:1005A0008A420DD80DE0DDF81210B1F5F42F00D914
:1005B000A570DDF81610C1F30B41B1F5107F00D026
:1005C000A570012803D0022801D0052839D10222C4
:1005D00006F21D4168460097FFF760FF00990298F8
:1005E00089B2884200D0A570012206F225416846F2
:1005F0000097FFF753FF0099BDF80500C9B2884284
:1006000000D0A5709DF8040002281AD1042206F239
:10061000494168460097FFF741FFDDF81600009951
:10062000884200D0A570012206F24D41684600972D
:10063000FFF734FF00989DF80710C0B2814200D048
:10064000A5709DF81C00401EFE2800E01FE000D2AF
:10065000A570BDF80500A0F57F41FF3901D03F2806
:1006600002D19DF8070020B901A8FFF74BFF00B9A0
:10067000A570DDF812001B36064401A8FFF742FF03
:1006800030B1E07880B1217988420DD012E0A570B8
:100690009DF81C0010B92079401C2071E078401CA6
:1006A000C0B2E0700C2801D3A57003E0A078002848
:1006B0003FF442AFA07808B0BDE8F081303132336A
:1006C000343536373839414243444546000000103E
:1006D00038010010F44D0000FE4910B5486980044F
:1006E0000CD4FD4A906843F698239468241A9C42DF
:1006F000FBD34869800401D4012010BD052000F01F
:1007000075FE002010BD70B5F34CA668042000F003
:100710006DFEF24D03E000BFFFF7DEFF48B1A068B9
:10072000801BA842F8D308E0FFF7D6FF08B10120EC
:1007300070BDA068801BA842F6D3002070BD2DE9D3
:10074000F041092000F052FEE54800264FF47A7788
:100750000670C821384601F080F9DF4CA06842F2EB
:100760001075A168091AA942FBD3C821384601F0C7
:1007700074F9A068A168091AA942FBD3C8213846B8
:1007800001F06BF9D748022186708171C670BDE80F
:10079000F0818AB046208DF814004FF000098DF8E2
:1007A000179036208DF81500CF4A33208DF81600AB
:1007B0001068CA464FF6FF031840CC4B40F48070D7
:1007C00018431060CA48CC49CE4DC0F80090C948C3
:1007D0000068A0F56C50FF380860C84900F5E0508B
:1007E0000860C749400A0860F8202870FF20687038
:1007F000A87001F0F5F8BB4CC34A002094F905102D
:1008000052F821102A1802F580520B5C401C82F825
:1008100000386028F6D34FF4E175294640F24910BC
:1008200001F01BF9294640F29F1001F016F94FF430
:10083000005BDFF8D8825D46207808B101F0D6FD74
:10084000A07928B1012818D02078002879D0FFE0BD
:100850000A2000F0CBFDFFF761FE10B1FFF76FFF3C
:10086000EAE70120A0715D4684F803A0062000F0AD
:10087000BDFD0A2000F0BAFDDEE719222946A34893
:10088000FFF70CFE98F8180000287CD098F80000BC
:10089000062873D2DFE800F072030B46464940F2A7
:1008A000044000880390D8F80410814266D098F87C
:1008B00009104FF00109404601295FD1D0F80A1014
:1008C00019B993498969C0F80A100026804617E0D3
:1008D000072000F08BFDD7F80E00B846871B402F8D
:1008E00000D94027A9193A468A481931FFF7D6FDA1
:1008F000D8F80A003A4630448649FFF777FC3E4470
:10090000D8F80E004746B042E2D83978012935D1EF
:100910004FF0E0220906C2F88011D7F80A00FFF76D
:1009200093FC2BE04FF001092BE098F809104FF0F1
:100930000109032925D16F49774A00260B68136006
:1009400017E07EE0072000F051FDD7F80E00871B6E
:10095000402F00D94027A9193A466E481931FFF7B0
:100960009DFD64483A46006881196A48FFF785FD95
:100970003E44D8F80E004746B042E3D898F8180035
:1009800008B1464600E01CE098F80800C00613D500
:100990006149012203A8C1F800B005F11801CDF8A2
:1009A0000CA0FFF75BFD307820B1C8214FF47A70BE
:1009B00001F053F8307E20B1307A800701D5FFF77F
:1009C00071FCD8F80E001B3505445048FFF79AFD1E
:1009D00048B302204249A0715D4681F800A00B2077
:1009E00000F004FDB9F1000F1DD03B484FF00009A5
:1009F000816842F2107283685B1A9342FBD34FF412
:100A00002F714FF47A7001F028F832494869400399
:100A100005D5486D400502D50020099001E00998F0
:100A200008B9FFF73FFCE078401CC0B2E0700C282A
:100A300002D30120A07011E7A07800283FF410AF86
:100A40000CE70120207001F065FB012001F023FB81
:100A5000234800780028F1D0002105A800F027FCE9
:100A60000028EBD084F806A05D4684F803A0E3E6F6
:100A70001C4C0026FF202660A680A671607100F045
:100A8000EEFD00F043FEFFF763FC00F075FC002074
:100A900000F0ACFC01F006FD0E4F7869400302D572
:100AA000FFF71AFED0B3042000F0A0FC78690A4DCD
:100AB00080043AD4FFF727FE80B3FFF724FE68B323
:100AC000FFF721FE50B3042000F090FCA868034912
:100AD0007A6924E0008009200000094080841E001B
:100AE0007C0000100C0000100CED00E00000FA0586
:100AF000C000001008000010B0000010A800001096
:100B0000AC0000109101001074000010780100107A
:100B10007C4D000038010010000000100DE0920430
:100B200003D4AA68121A8A42D2D3A86842F210717A
:100B3000AA68121A8A42FBD36671FFF781FCFFF79D
:100B4000EDFC80B1FFF787FB68B1022000F04EFC9E
:100B500094F90500401C03D10C488069FFF774FB31
:100B60000120607004E0022000F040FC66706671B5
:100B7000FFF7B2FD40B140210548FFF732FC4022AB
:100B8000D1010348FFF779FCFFF703FE7C4D00001D
:100B9000380100102DE9F047FE4A00234FF400779A
:100BA000156A4FF4FF79C5F30724DFF8ECA34FF47F
:100BB000E05CDFF8E883FA4E25E0B84216D213284D
:100BC0000CD014280CD048450CD0A0F58072FF3A08
:100BD0000AD03E2813D81AF8002011E0EAB20FE03C
:100BE00022460DE055220BE0AA2209E0604506D21C
:100BF00008EB0002A2F5805292F8002E00E00022DD
:100C0000F254401C5B1C8B42D7D3BDE8F08770B513
:100C1000E04D2C6B402C00D94024E86AE9690219A8
:100C20008A4202D90C1A042169702146FFF7B2FFEB
:100C30002246DB49822001F02EFBE86A2044E8626C
:100C4000286B011BD74829638268A2EB04028260EB
:100C500005D06978022901D00021017370BD0321FC
:100C60006970F9E7CF4910B5CF4808600D2282209E
:100C700001F011FBC7490520487010BD70B50D4645
:100C8000CA494A69520302D5496D490521D4B0F5D4
:100C9000007F1ED3C64BBF4CB0F5E05F1AD29968F7
:100CA000A269891AC34A914204D39968A1610021BB
:100CB00061606161BB4A00215F3AB84B07E04418AC
:100CC0001C44565CA4F58054491C84F8006EA9426B
:100CD000F5D370BD616921B99968A16199686161B5
:100CE000A060B54949790029F3D199686269891AE8
:100CF000B24A91421CD2B24A012111709968A16195
:100D000099686161A168401A6168884203D9616A83
:100D1000884200D26060062000F068FB61682A46C5
:100D2000BDE870409F4801F500515F38FFF7A5BB53
:100D3000BDE870400C2000F059BB10B5954CA1786F
:100D4000E06A4218E1698A4206D9081AA0700520B3
:100D50006070022001F05AFAA178E06AFFF78EFF76
:100D6000A178E06A0844E062206B421A8D48226351
:100D70008368A3EB0101816002D06178052904D169
:100D800000210173BDE810406CE710BD2DE9F04172
:100D9000804CA178E06A4218E1698A4206D9081AB3
:100DA000A07005206070022001F030FA7D4D002116
:100DB000A0787B4B5F3DE26A08E056186F5C9E5D51
:100DC000BE4202D00021A16202E0491C8142F4D35C
:100DD0001118E162216B0A1A724922638B68A3EB36
:100DE0000000886002D06078052808D1A06A20B190
:100DF00000200873BDE8F04134E70120F9E7BDE8C1
:100E0000F081684810B51F38D0F81110027D09BA7A
:100E100021F0FF0111435F4A4902D162C18A49BAF8
:100E200049021163806888420CD0822001F0EEF9FB
:100E3000022001F0EBF95B4902200873FFF712FF73
:100E4000002010BD012010BD70B55648554D1F380B
:100E50000224816829B1007B000607D4022001F03A
:100E6000D5F92C73FFF7FEFE002070BD012070BD88
:100E700010B54C48474C1F388068A178884200D292
:100E8000A0704849A2785F39822001F004FA03205B
:100E900060704448A2788168891A816000210173DA
:100EA00010BD404810B51F38816839B1007B00067D
:100EB00001D5822000E0022001F0A8F93949002084
:100EC0000873BDE81040CDE610B5FFF7BDFF002860
:100ED0001FD0344870215F38022201700021417018
:100EE0008270C1700171417181710A22C2710172F7
:100EF00041728172C1723022027301224273817386
:100F0000C17301744174234912208870BDE81040F8
:100F1000AEE710BD1CB5FFF797FF00286AD029483F
:100F20000A22062103886846FFF76EFA1D48002250
:100F30005F3880230270437082700121C1702021CC
:100F4000017143718271C271412202725422427254
:100F50004F2282724C22C272017341738173C1733A
:100F60004622027450234374722383746923C3742A
:100F70006E230375742343758175C2756C220276E6
:100F800061224276732282766822C27601774177A7
:100F9000817719E08C0000103C4D00009101001099
:100FA00038010010F01B00105553425300800920F7
:100FB00000000940A08601000C00001020A10700DD
:100FC0007C00001004040000C1779DF8011080F837
:100FD00020109DF8021080F821109DF8031080F871
:100FE00022109DF8041080F82310DF492420887017
:100FF000FFF73EFF1CBD10B5FFF726FF00280CD001
:10100000DA4803210170002141708170C170D64916
:1010100004208870BDE810402AE710BD10B5FFF726
:1010200013FF002810D0D148002106220170427021
:101030008170C170017141718171C171CA4908200B
:101040008870BDE8104013E710BD10B5FFF7FCFE37
:10105000002815D0C44AC548116A491E0B0E0370FA
:101060000B0C43700B0A8370C17000210171417138
:1010700002238371C17108209070BDE81040F7E62B
:1010800010BD10B5FFF7E0FE002819D0B7480021C9
:10109000B54B0170417081700822C2701A6A140E3B
:1010A0000471140C4471140A8471C2710222027218
:1010B00041728272C1720C209870BDE81040D7E670
:1010C00010BD2DE9F041A84DA84C0021A87840346E
:1010D000A64A02E0535C6354491C03468142F9D39B
:1010E0001F2B72D12068A24988426ED19F4E606842
:1010F0005F364FF001087060A068B060607B18B97F
:10110000A07B08B1102802D986F80C8059E0E07B5A
:101110001E28F9D00FDC12282ED005DC48B3032896
:10112000F2D1BDE8F041CFE61528EDD01A28EBD179
:10113000BDE8F0415FE702272A2828D010DC2328E9
:101140001DD025281ED02828DED1FFF75AFE002802
:1011500026D0207B000618D56F70BDE8F04156E51B
:101160002F281ED05528CFD05A28CDD1BDE8F04128
:1011700054E7BDE8F04194E6BDE8F041CAE6BDE8B9
:10118000F0417EE7BDE8F0415FE7022016E0FFF79F
:1011900038FE002804D0207B00060ED485F801809C
:1011A0002DE6FFF72EFE0028FAD0207B000604D49F
:1011B00085F80180C5F8288021E6822001F026F814
:1011C0003773BDE8F0414DE5FFE7822001F01EF8DE
:1011D000022001F01BF80620687010E6624810B586
:1011E0004178022908D003290ED004290FD00529FF
:1011F00001D10021417010BD5C484030C07B2828DF
:10120000F9D1BDE8104002E5BDE810402AE5822092
:1012100000F0FCFFF8E710B55449022001F00AF88D
:1012200051498870487858B101280CD0022000F04C
:10123000EDFF4E4902205F310873BDE8104011E513
:10124000BDE810403DE749484030C07B2A2804D023
:101250002F2805D1BDE8104098E5BDE810406CE5A9
:1012600010BDFFB50246002002EB420501464FF4D7
:1012700040566C4603AA6B1844F82130B34202DD95
:10128000002004B0F0BD3B4F07EB6307DB073F785E
:10129000575401D03B095354535C8F0003F00F03A4
:1012A0005354BB40491C18440329E4DBE9E7F0B57B
:1012B00006460020034602462E4C4FF4007700E01D
:1012C0005B1CF55C45B102EB030CA4440CF5805C9F
:1012D0009CF800C8AC45F3D0032B40D302F5C050B6
:1012E0002044037F457FC67F03EB0523857F2D04C4
:1012F00005EB06652B4451EA03052CD021B91A49A8
:10130000496840318B4226D8184B00216C33551860
:10131000254405F5805595F800585D54491C0C2965
:10132000F5D3817EC27E01EB0221027D407D120455
:1013300002EB00600C182046FFF793FF40F6F575AE
:1013400002E000BFFFF78DFFC11EA942FAD3A0F54E
:101350007061FF3901D00020F0BD2046F0BD203281
:10136000BA42AED3F0BD00008C000010911B0010FB
:101370005553424391010010002070476949C2074C
:1013800002D04FF000728A67800702D54FF080606C
:101390008867002070476349C20702D04FF000728F
:1013A000CA67800702D54FF08060C8670020704789
:1013B000014600205B4ACB0703D0536F9B0100D549
:1013C0000120890704D5516F490101D540F0020081
:1013D000704710B50446FFF7EBFF0346FFF7DBFF4E
:1013E00024EA0300FFF7CAFF002010BD70B54E4B82
:1013F00050B15968042403250226052907D2DFE8E5
:1014000001F0072B4A718E0000205860986070BD73
:10141000042807D0052809D0012402287AD0012801
:1014200008D00FE00320FFF7B6FF46E0BDE87040AC
:101430000120B0E70320FFF7AEFF0BE0FFF79EFFB0
:101440005C6070BD0E28FCD10320FFF7A4FF0220D2
:10145000FFF794FF0120F1E706280AD0032810D0F7
:101460000A2813D0092811D00D280FD00C28D9D064
:1014700070BD0320FFF78FFF0220FFF77FFF5E6044
:1014800070BD0320FFF787FF012027E00320FFF74F
:1014900082FF022012E0062813D00A281AD0092859
:1014A000C8D00C28BED00D28F0D00F28E8D10320DA
:1014B000FFF771FF0220FFF761FF0120BDE87040D8
:1014C0005CE7986810F01F0F00F101009860D7D119
:1014D00002201BE00320FFF75EFF0220FFF74EFF14
:1014E0005D6070BD072806D00A289BD00B2811D05C
:1014F00009289FD070BD0220FFF74DFF986810F0BB
:101500003F0F00F101009860F4D10120BDE8704068
:101510005FE7FFE70320FFF73EFF02208EE7062884
:10152000A7D08FE700800920D0000010F0B57248E6
:10153000D0F804114FF00002CB05704928D4D0F840
:101540000C31DC076E4B03D0D0F8A041640660D5A7
:10155000D0F80441E40605D0D0F8044104F01F049B
:10156000B3FBF4F40C60D0F8A851ED060ED0D0F81F
:10157000A85105F01F05B3FBF5F34B60D0F800311F
:1015800003F001035B1CB4FBF3F331E00023F4E749
:10159000D0F88830DB053CD5D0F80C31DB0703D020
:1015A000D0F8A0315B0634D5D0F88830D0F80441AB
:1015B00003F01F0314F01F05D0F8A841D0F8006114
:1015C00004F01F0406F0010603F1010306F1010611
:1015D00003D04B4F5F43B7FBF5F50D6024B1484F87
:1015E0007B43B3FBF4F300E000234B60B5FBF6F361
:1015F000C1F80830D0F80831DB05D0F808311CD527
:1016000013F01F0303D0042B07D0062B05D0CA60AC
:10161000F0BD0A604A608A60ECE7D0F88820D0F814
:10162000083102F01F02D0F80C0103F01F03344808
:10163000521C4243B2FBF3F00FE09B05E7D5D0F814
:101640000C21D20702D0D0F8A80001E0D0F8880021
:101650002B4A00F01F00401C5043C860F0BD2648D4
:1016600010B42021C0F8A011D0F8A0114906FBD574
:101670000121C0F80C110922C0F88420C0F88010A4
:10168000AA22C0F88C205523C0F88C30D0F88840AE
:101690006405FBD52324C0F8A440C0F8A010C0F80E
:1016A000AC20C0F8AC3000BFD0F8A8205205FBD564
:1016B00040F20112C0F8042140F20122C0F80821D2
:1016C000C0F800110221C0F8B4110421C0F8A8111B
:1016D0000C49C0F8C4100021C0F8C811D0F8B021DE
:1016E00042F00302C0F8B02145F23A020260064817
:1016F000016010BC1AE7000000C00F40DC000010C1
:10170000001BB700FE9FF8F708ED00E0F0B5AE490A
:10171000032008630020C1F80801AC480422826558
:10172000026C42F004020264A94A8A6600220A613D
:101730001022C261026822F0100202600322C1F886
:101740007022C1F8742200224A644FF40032826190
:10175000026842F4003202600922C1F80021C1F897
:1017600004211022C1F8D42052048263026A42F498
:10177000001202620D22C1F8D020C1F8E020002240
:10178000C1F8F4204FF00052C263026A42F00052E6
:1017900002620022C1F8F0204FF08052C263026A58
:1017A00042F0805202621022CA670204826102681B
:1017B00042F0004202601022C1F814212027876500
:1017C000026C42F0200202641022C1F81C21802227
:1017D000C265026C22F0800202649026C1F8FC60AF
:1017E0000204C263026A22F0004202621022C1F8BF
:1017F000DC20D204C263026A22F4000202620122E7
:101800000A66CA654A660323C1F8D8300523C1F8C1
:10181000E4308A601123CB60CA630B640224C1F8F0
:1018200020411225C1F824510C604D600C604D60C0
:1018300010248C659405C461046844F48004046039
:101840000124CC630B641023C1F82C31CB14C36585
:10185000036C43F4006303641023C1F830318B142C
:10186000C365036C43F48053036440F282234B62EC
:101870009A240C62CB6110234B618761036843F0AB
:101880002003036010238B6140248461036843F0CC
:101890004003036001230B67CB6640F20243CB6237
:1018A0008B621023C1F8E83093068363056A45F024
:1018B000806505621025C1F8EC50D506C563056A40
:1018C00025F0006505624E635503C561056825F482
:1018D000005505600025C1F8E851C367036E43F069
:1018E00080630366C1F8E4515306C367036E43F097
:1018F000007303668A23C1F8F8300823C1F8C830A2
:101900009504C563066A46F4802606621026C1F86F
:1019100028610E15C665066C26F4806606640126ED
:10192000C1F88060C1F88460C1F89060C1F8A0601F
:10193000C1F8A460C1F8A860C1F8B860C1F8BC6083
:10194000C1F8C060C1F8C4600026C1F81861C46560
:10195000046C44F0400404640B651405C46104681D
:1019600024F480140460CB64D404C461046824F4B7
:10197000002404608B64C561046824F4802404603E
:101980000024C1F80C418365036C43F00803036431
:10199000C1F8104110238365036C43F01003036406
:1019A0000C480D4B0068984204D141F8B82F8A606A
:1019B000CA60F0BD094A9042FBD1812041F8B80FBE
:1019C0008860C860F0BD000000C0024000800920AF
:1019D00002000100CC000010473F1927473F19477C
:1019E000374800210167C1600222426181613022D3
:1019F000C263344882683448C0E900210846704711
:101A000070B541F28832904215D8642800D290B95E
:101A100042F2107291420ED805290CD3294CA268CB
:101A2000294B1D68521B5D6805EB4506C6EBC515C5
:101A3000B2EBC50F01D2002070BD214A02255560CE
:101A400038B1224EB6FBF0F0401090615560012095
:101A50005060A068C3E90001EDE770B51A4C00259D
:101A60000E466560FFF7CCFF164A06EB460120687C
:101A7000C1EBC61193681B1AB3EBC10FFAD3104820
:101A800002214160C16B01F0FE01C163002065606D
:101A900070BD0C4880680C490A68801A4A6802EBDD
:101AA0004203C3EBC212B0EBC20F08D304480222B8
:101AB0004260C26B02F0FE02C263002048607047C1
:101AC0000080004000000940F000001080C3C90100
:101AD000FA4800214FF00112818001704170C0E985
:101AE00002217047F5491C31002000F0A3BB10B55E
:101AF000F24C1434A288402A00D940228020216868
:101B000000F0C9FB216801442160A188081AA08067
:101B100010BD10B5E94C00201434216800F08AFB98
:101B2000216801442160A188081AA08010BD00220C
:101B30001146802000F0AFBBE149002000F07ABBE5
:101B400070B5DE48DD4D1C3005F11405007810F04D
:101B50001F040AD0D949DA4B01F11C004A780079F8
:101B6000012C06D0022C26D109E0D448001D2860A3
:101B70001DE002B3897888421DD2002015E000F0F4
:101B80008F04200605D504F00F064FF48030B040D6
:101B900001E00120A0400AB922070CD18A68024264
:101BA00009D0C9680142E8D0012018802B60FFF7F6
:101BB0009EFF012070BD002070BD024670B5BF4879
:101BC000BE4C1C30017811F01F030146498804D037
:101BD000012B29D0022B27D111E0012924D132B1C8
:101BE000012000F0C2FAA08840F0020005E00020C9
:101BF00000F0BBFAA08820F00200A08021E000796C
:101C000000F08F00030605D500F00F034FF4803578
:101C10009D4001E00125854063782BB1030703D087
:101C2000A3682B4200D009B1002070BD22B100F0A2
:101C3000EDFAE068284303E000F0F2FAE068A84318
:101C4000E060012070BD9D4810B51C30007810F098
:101C50001F0F9A4800F11C00C0782AD1974914310F
:101C6000012807D001F108020228937806D0032842
:101C70001FD112E093480860122012E0924800221F
:101C800004E004780CB144882044521C9342F8D1FB
:101C9000027872B10860408803E08C4818440860FC
:101CA00000788A88824200D98880FFF720FF0120CF
:101CB00010BD002010BD2DE9F84F804F00201C37CB
:101CC0000090B8787D4E4FF000094FF0010A4FF4B4
:101CD000803B00286BD07C4C65E06078022804D003
:101CE000042841D005285CD141E06179B87881426F
:101CF00038D170702079B0707049002011F1100156
:101D000001F80090401C0428FAD301254FEA060888
:101D10000AFA05F0D8F80810084202D0284600F068
:101D200061FAD8F808100BFA05F0084203D045F024
:101D3000800000F057FA6D1C102DE9D34FF0011010
:101D4000C8E90209012000F011FAE0794006B8F86C
:101D5000040002D540F0010001E020F00100A8F8E5
:101D600004001EE060881DE0E078009019E0009813
:101D7000B8B9A07800F08F05280604D505F00F014A
:101D80000BFA01F001E00AFA05F0B16801432046C0
:101D9000B16000F000FA284600F01AFA284600F078
:101DA0002BFA207804442078002896D11FE086F88A
:101DB000019001245546D846B16805FA04F008425E
:101DC00002D0204600F00EFAB16808FA04F008428A
:101DD00003D044F0800000F005FA641C102CEBD313
:101DE0004FF00110C6E90209002000F0BFF9B878F1
:101DF0007178884202D10120BDE8F88F0020FBE70E
:101E00002DE9FC5F2D4D00273E466878BB46B8465D
:101E1000002871D0BA462C4C05F11C0968E06078A6
:101E2000022804D0042808D005285FD119E0607981
:101E3000697888425AD0608859E0A77899F80410E8
:101E4000E6784FF00008B94250D199F80200B0424C
:101E50004CD11A484FF0010A103010F807B0C6559F
:101E600044E099F80410B94240D1A17801F08F0103
:101E70000191090605D5019901F00F024FF4803157
:101E800001E0019A01219140009199F80200B042CD
:101E90001ED1A8680843A860E968009881432046DD
:101EA000E96000F078F9019800F092F9019800F0EB
:101EB000A3F9009948EA010818E00000F8000010B2
:101EC000341D00106C4E00007E4E00009F4E00003E
:101ED0005E450BD118EA010F08D1A8688843A860B5
:101EE000E8688843E860019800F07CF920780444B1
:101EF0002078002893D15046BDE8FC9F2DE9F041A1
:101F0000494C0027A4F108062178A4F11C050828F3
:101F100063D2DFE800F06204647262628381FFF7DB
:101F2000E1FD2078C00900F052F9E088B080207807
:101F3000C0F34111F1BB61780C294AD2DFE801F00E
:101F40000609490B49101A1D1F253142FFF7F8FDFC
:101F50004DE0002000E00120FFF72FFE50B306E027
:101F600010F01F0F35D1A07840F080002870BDE838
:101F7000F041DCE5FFF767FE39E000202AE010F0D1
:101F80001F0F26D128481B381AE010F01F0F20D150
:101F9000FFF791FE70B1FFF7CAFDBDE8F04100F018
:101FA0006DBA00F01F00012813D1687810B12079B4
:101FB000A97800E00DE088420BD21B490C39084497
:101FC00030601CE000F01F00012802D1FFF718FF6D
:101FD000C4E7802000F01AF9B780BDE8F081080658
:101FE00008D4B0880028F8D0FFF793FDB088002807
:101FF000EFD0F2E7BDE8F0419EE5080602D5BDE866
:10200000F04174E528780106E7D500F07F002870DC
:10201000BDE8F04100F054B8802000E00020BDE8A9
:10202000F04100F0FDB80000140100100146000767
:10203000C00E090600D5401C7047DC491022C1F8CB
:102040000822C1F8100200BFD1F80002C006FBD57B
:102050007047D64A1023C2F80832C2F8100200BFF7
:10206000D2F80002C006FBD5C2F80832C2F810123E
:10207000D2F80002C006FBD57047CC493022C1F827
:102080000822C1F8100200BFD1F800028006FBD57B
:10209000D1F81402704710B5040001D0012000E00F
:1020A00000204FF4807141EA0041C148FFF7D1FFA1
:1020B000C0494FF480200CB1886310BDC86310BDC7
:1020C00030B5BD49BD4D41EA004421462846FFF7E1
:1020D000C0FF21462846BDE83040BAE7B34800219A
:1020E000C0F848124021C0F84C120122C0F8482222
:1020F000C0F84C12D0F80012C905FBD54FF0FF31E3
:10210000C0F83812C0F83412C0F808120C21C0F818
:102110000412704730B5AA4C1A202060221D1168A5
:1021200030EA0101FBD1A74901234B678B679F4D23
:102130000023C5F810318A23C1F8F83020601168F7
:1021400030EA0101FBD14FF0E0214FF08070C1F87F
:1021500080029D4B202283F80024C1F80001FFF784
:10216000BDFFBDE830400020AAE7704710B500B1C0
:1021700001204FF4807444EA00419448FFF769FF5E
:102180008A480321C0F84412D0F80012C905FBD5D3
:10219000C0F8084210BD10B502468078FFF746FF30
:1021A0008249D1F84432012484402343C1F84432A7
:1021B000C1F848029088C1F84C0200BFD1F8000273
:1021C000C005FBD54FF48070C1F8080210BD704700
:1021D00000B5FFF72BFF7E495DF804EB41EA0040B4
:1021E000891336E700B5FFF721FF79495DF804EB65
:1021F00041EA004077492CE700B5FFF717FF744923
:102200005DF804EB41EA0040891322E700B5FFF7CF
:102210000DFF6F495DF804EB41EA00406E4918E795
:1022200000B5FFF703FF6A495DF804EB41EA00409F
:1022300089130EE700F00F02012370B503EB820350
:102240005A4AC2F8283200BFD2F820321C05FBD50A
:10225000C3F309030024DD1C05E000BFD2F81862B7
:1022600041F8046B641CB4EB950FF7D30021C2F85E
:10227000281241F24821C140C9070AD1FFF7D6FE12
:102280004FF4A06141EA0040FFF7D7FE5348FFF743
:10229000D4FE184670BD70B513460546434C00F099
:1022A0000F00022202EB8000C4F82802C4F8243296
:1022B0000020DA1C05E000BF51F8046BC4F81C6272
:1022C000401CB0EB920FF7D30020C4F82802284638
:1022D000FFF7ACFE4FF4A06141EA0040FFF7ADFE0E
:1022E0003F48FFF7AAFE184670BD2DE9F0412F4D7B
:1022F000D5F80032C5F80832180721D52C48FFF769
:102300009CFE3848FFF7B9FEC10605D5FFF7E6FE8B
:10231000BDE8F04100F0A3B8810705D5BDE8F04164
:1023200000F0010000F095B8010709D5400703D57A
:10233000BDE8F04100F09AB8BDE8F04100F09DB86A
:10234000294E58074FF001071CD4BDE8F081002446
:10235000D5F8302207FA04F10A4210D06008C5F817
:10236000381200BFD5F800128906FBD5D5F8141233
:10237000E2070CD056F8201009B103208847641CEE
:10238000202CE5D3D5F830020028E0D1DDE73CB9B8
:10239000490705D5316819B1012088470124D7E7DD
:1023A00056F820100029EAD00220E7E700C00820F4
:1023B0000005FE0000800920000180000005D0001B
:1023C000F4CF082000C0024018E000E00005D8006B
:1023D0000005400000012000000101000005F2009E
:1023E0000005FA000002FE00104F000070B5284CF6
:1023F000607820B30026274D012810D002280DD187
:10240000A8686168401A2449884215D32348406B64
:10241000400011D50120FFF73EFE667070BDA86830
:102420006168401A1E498842F8D30020FFF733FE46
:10243000A86860600220607026700C2005E020789B
:102440000028EBD1012020700D20BDE87040FEF780
:10245000CDBF002802D10E4901204870704710B549
:10246000FFF736FB0A490020487010BD08480121DB
:102470004170084989684160704770477047022879
:1024800003D0032803D1FEF7A9BEFEF7C4BE7047F0
:102490001C01001000000940A086010000800920F6
:1024A00040420F0019480621016107210160002107
:1024B0004161416202214160C168C906FCD400E06B
:1024C0008168C1684907FBD4002070470F498860C4
:1024D000C868C006FCD48868704700B50B46024641
:1024E00004E000BF12F8010BFFF7F0FF5B1EF9D20A
:1024F00000BD00B50B46024604E00020FFF7E6FFF2
:1025000002F8010B5B1EF8D200BD00000000034082
:102510002DE9F047F84E80464FF080773068402430
:10252000F64DB84249D100BF00BF00BF00BF00BF99
:1025300000BF00BF00BF00BF00BF00BF00BF00BFA3
:1025400000BF00BF00BF00BF00BF00BF00BF00BF93
:1025500000BF00BF00BF00BF00BF00BF00BF00BF83
:1025600000BF00BF00BFEC611520FFF7AFFF0020E8
:10257000FFF7ACFF00F0FF09AC6100BF00BF00BF78
:1025800000BF00BF00BF00BF00BF00BF00BF00BF53
:1025900000BF00BF00BF00BF00BF00BF00BF00BF43
:1025A00000BF00BF00BF00BF00BF00BF00BF00BF33
:1025B00000BF00BF00BF00BF00BF00BF00BF00BF23
:1025C00000BF00BF00BF00BF00BF00BF00BF00BF13
:1025D00000BF00BF00BF00BF00BF00BF00BF00BF03
:1025E00000BF00BF00BF00BF00BF00BF00BF00BFF3
:1025F00000BF00BF00BF00BF00BFEC610620FFF7B7
:1026000065FFAC6100BF00BF00BF00BF00BF00BFDF
:1026100000BF00BF00BF00BF00BF00BF00BF00BFC2
:1026200000BF00BF00BF00BF00BF00BF00BF00BFB2
:1026300000BF00BF00BF00BF00BF00BF00BF00BFA2
:1026400000BF00BF00BF00BF00BF00BF00BF00BF92
:1026500000BF00BF00BF00BF00BF00BF00BF00BF82
:1026600000BF00BF00BF00BF00BF00BF00BF00BF72
:1026700000BF00BF00BF00BF00BF00BF00BF00BF62
:1026800000BF00BFEC610120FFF720FF4FEA880088
:10269000FFF71CFF3068B84202D14846FFF716FF2B
:1026A000AC6100BF00BF00BF00BF00BF00BF00BFE4
:1026B00000BF00BF00BF00BF00BF00BF00BF00BF22
:1026C00000BF00BF00BF00BF00BF00BF00BF00BF12
:1026D00000BF00BF00BF00BF00BF00BF00BF00BF02
:1026E00000BFBDE8F0872DE9FC5F8846044601A9DC
:1026F000834800F05AFB834D834E844FF0BB032088
:102700008DF8000020098DF8010020018DF80200ED
:102710004FF000098DF8039000BF00BF00BF00BF5D
:1027200000BF00BF00BF00BF00BF00BF00BF00BFB1
:1027300000BF00BF00BF00BF00BF00BF00BF00BFA1
:1027400000BF00BF00BF00BF00BF00BF00BF00BF91
:1027500000BF00BF00BF00BFDFF8A0B14FF0400ACC
:10276000CBF81CA004216846FFF7B7FE0024002028
:10277000FFF7ACFEC0B28DF8040000E003E018F8EB
:102780000410884208D082202860222030607846D9
:1027900038608220BDE8FC9F641CB4F5805FE6D3FE
:1027A000CBF818A000BF00BF00BF00BF00BF00BF34
:1027B00000BF00BF00BF00BF00BF00BF00BF00BF21
:1027C00000BF00BF00BF00BF00BF00BF00BF00BF11
:1027D00000BF00BF00BF00BF00BF00BF00BF00BF01
:1027E00000BF00BFC5F800907846C6F8009038607A
:1027F0000020CFE72DE9F0474FF0000900BF00BFF0
:1028000000BF00BF00BF00BF00BF00BF00BF00BFD0
:1028100000BF00BF00BF00BF00BF00BF00BF00BFC0
:1028200000BF00BF00BF00BF00BF00BF00BF00BFB0
:1028300000BF00BF00BF00BF00BF00BF40252F4E3C
:10284000F5619F20FFF742FE0020FFF73FFE00F0FA
:10285000FF080020FFF73AFEC4B20020FFF736FE63
:10286000C1B2B56100BF00BF00BF00BF00BF00BF65
:1028700000BF00BF00BF00BF00BF00BF00BF00BF60
:1028800000BF00BF00BF00BF00BF00BF00BF00BF50
:1028900000BF00BF00BF00BF00BF00BF00BF00BF40
:1028A00000BF00BF174D184E184FB8F1C20F01D12D
:1028B000202C07D0822028602120306078463860A4
:1028C00082200EE70C48142912D0152920D0162991
:1028D00022D0182923D0C0F800900020FFF718FE5E
:1028E000C5F800907846C6F8009038600020F8E6F9
:1028F0004FF480110EE00000240100100080092038
:10290000A0860100800000108400001088000010E4
:102910004FF400110160E0E74FF48001FAE74FF057
:102920008071F7E72DE9F34FC3B0804600244FF0E4
:10293000820AFE4DFE4EFF4F4FF0210BA14641A9EA
:10294000FD4800F032FA00286AD100F099FA02201E
:102950008DF800004FEA18108DF8010004EB081004
:102960008DF8020044988DF8039000EB04214FF499
:10297000807201A8FDF71CFD00BF00BF00BF00BFB3
:1029800000BF00BF00BF00BF00BF00BF00BF00BF4F
:1029900000BF00BF00BF00BF00BF00BF00BF00BF3F
:1029A00000BF00BF00BF00BF00BF00BF00BF00BF2F
:1029B00000BF00BF00BF00BF4020E049C8614FF426
:1029C00082716846FFF789FDDC494020886100BFBD
:1029D00000BF00BF00BF00BF00BF00BF00BF00BFFF
:1029E00000BF00BF00BF00BF00BF00BF00BF00BFEF
:1029F00000BF00BF00BF00BF00BF00BF00BF00BFDF
:102A000000BF00BF00BF00BF00BF00BF00BF641C0D
:102A1000E4B2102C93D341A9C74800F0C6F948B1DD
:102A2000C5F800A07846C6F800B03860822045B0EE
:102A3000BDE8F08F00F06DFAC5F800907846C6F852
:102A4000009038600020F2E72DE9F04F89B0DFF800
:102A5000DC825FEA020B4FF0000607910FD04FF4C3
:102A6000805501462A466846FDF737FCDDE90047F8
:102A7000284601F02DFF5FEA00090CD016E0862100
:102A8000AB48C8F80010092101607946A9480160E7
:102A9000862009B0CCE78221A548C8F80010222181
:102AA00001607946A34801608220F2E7ABEB06059E
:102AB000C7F580504FF0000AA84200D20546B5F590
:102AC000805F04D02046494600F09DFCD8B90798A5
:102AD0002A46811907EB0900FDF76AFC204600F041
:102AE00018FC80B920464946FFF71CFF58B920461C
:102AF0004946FFF7F8FD78B10AF1010000F0FF0A3E
:102B0000BAF1030F05D3484601F0BAFED8F8000029
:102B1000BFE7BAF1000FE1D12E440027641C5E45E7
:102B2000C4D3484601F0ACFE81490020C8F800003B
:102B3000086079467F4801600020AAE72DE9FF4F31
:102B40008DB00D46DDF868900026784C07935FEA5B
:102B500009013ED04FF4805701463A466846FDF7DA
:102B6000BCFBDDE900B10C913A46691C6846FDF7F3
:102B7000B4FBDDE90010CDE904013A4668460F993F
:102B8000FDF7ABFBDDE90085A9EB0607C5F5805035
:102B9000B84200D2074625B1D8457CD10C98854271
:102BA00079D14FF4805001F093FE5FEA000A1BD008
:102BB000D8454FD10C9885424CD12A464FEA08306F
:102BC000514600F0FAFA000618D5504601F058FEBA
:102BD00079E08620206056480921016078465549F1
:102BE0000860862011B023E782202060504822210F
:102BF000016079464F4801608220F3E705988045DF
:102C000009D1049901EB0030C1F58052514400F024
:102C1000D4FA0006D9D4404600F07BFB0006D4D499
:102C200007983A46811905EB0A00FDF7C1FBEA193E
:102C30004FEA0830514601F0D3F90006C5D4059992
:102C4000884533D1049800EB01300499C1F58052D6
:102C5000514427E0059988450AD1049800EB0130DA
:102C60000499C1F58052514600F0A7FA0006ACD491
:102C7000404600F04EFB0006A7D407983A4681195B
:102C80000F98304401F0ACF900069ED405998845B0
:102C90000CD1049800E00DE000EB01300499C1F57F
:102CA0008052514601F09CF900068ED4504601F046
:102CB000E7FD0AE007983A4681190F98304401F081
:102CC0008FF9000601D520688CE73E44002508F105
:102CD00001084E45FFF458AF1549002020600860F8
:102CE00078461449086000207CE715480068704762
:102CF0004FF4805070472DE9F04FDFF83080DFF857
:102D000030B089B00F0004464FF0000634D04FF4C5
:102D1000805501462A466846FDF7DFFADDE900A145
:102D200005912A46214606A80CE00000800000100C
:102D30008400001088000010A08601000080092097
:102D400024010010FDF7C9FADDE906404FF0000943
:102D5000BD1BC0F58051A94200D20D4620B154459B
:102D600015D10599884212D1204600F0D2FA00060A
:102D70000DD5D8F800008CE68621C8F8001009218E
:102D8000CBF8001079463B480160862081E62E444E
:102D9000641C4846BE42DBD3C8F800007946CBF835
:102DA000000034480160002073E62DE9F041324C08
:102DB0000F460646A56806E0A068401BB04202D355
:102DC0000120BDE8F081384600F003F80028F3D177
:102DD000F7E770B5044600BF00BF00BF00BF00BFEB
:102DE00000BF00BF00BF00BF00BF00BF00BF00BFEB
:102DF00000BF00BF00BF00BF00BF00BF00BF00BFDB
:102E000000BF00BF00BF00BF00BF00BF00BF00BFCA
:102E100000BF00BF00BF4025184EF5610520FFF739
:102E200055FB0020FFF752FB2070B56100BF00BFCB
:102E300000BF00BF00BF00BF00BF00BF00BF00BF9A
:102E400000BF00BF00BF00BF00BF00BF00BF00BF8A
:102E500000BF00BF00BF00BF00BF00BF00BF00BF7A
:102E600000BF00BF00BF00BF00BF00BF207800F060
:102E7000010070BD8800001000000940008009209A
:102E800070B500BF00BF00BF00BF00BF00BF00BFE4
:102E900000BF00BF00BF00BF00BF00BF00BF00BF3A
:102EA00000BF00BF00BF00BF00BF00BF00BF00BF2A
:102EB00000BF00BF00BF00BF00BF00BF00BF00BF1A
:102EC00000BF4025FB4CE5610620FFF7FFFAA56136
:102ED00000BF00BF00BF00BF00BF00BF00BF00BFFA
:102EE00000BF00BF00BF00BF00BF00BF00BF00BFEA
:102EF00000BF00BF00BF00BF00BF00BF00BF00BFDA
:102F000000BF00BF00BF00BF00BF00BF00BF00BFC9
:102F100070BD70B500BF00BF00BF00BF00BF00BFE5
:102F200000BF00BF00BF00BF00BF00BF00BF00BFA9
:102F300000BF00BF00BF00BF00BF00BF00BF00BF99
:102F400000BF00BF00BF00BF00BF00BF00BF00BF89
:102F500000BF00BF4025D74CE5610420FFF7B6FA5B
:102F6000A56100BF00BF00BF00BF00BF00BF00BF22
:102F700000BF00BF00BF00BF00BF00BF00BF00BF59
:102F800000BF00BF00BF00BF00BF00BF00BF00BF49
:102F900000BF00BF00BF00BF00BF00BF00BF00BF39
:102FA00000BF70BD70B5064600BF00BF00BF00BFC8
:102FB00000BF00BF00BF00BF00BF00BF00BF00BF19
:102FC00000BF00BF00BF00BF00BF00BF00BF00BF09
:102FD00000BF00BF00BF00BF00BF00BF00BF00BFF9
:102FE00000BF00BF00BF00BF4024B24DEC615020C5
:102FF000FFF76CFAAC6100BF00BF00BF00BF00BFAD
:1030000000BF00BF00BF00BF00BF00BF00BF00BFC8
:1030100000BF00BF00BF00BF00BF00BF00BF00BFB8
:1030200000BF00BF00BF00BF00BF00BF00BF00BFA8
:1030300000BF00BF00BF00BF00BF00BF00BF00BF98
:1030400000BF00BF00BF00BF00BF00BF00BF00BF88
:1030500000BF00BF00BF00BF00BF00BF00BF00BF78
:1030600000BF00BF00BF00BF00BF00BF00BF00BF68
:1030700000BF00BF00BFEC610120FFF727FAB000DE
:10308000FFF724FAAC6100BF00BF00BF00BF00BF64
:1030900000BF00BF00BF00BF00BF00BF00BF00BF38
:1030A00000BF00BF00BF00BF00BF00BF00BF00BF28
:1030B00000BF00BF00BF00BF00BF00BF00BF00BF18
:1030C00000BF00BF00BF70BD2DE9FE430F460446A0
:1030D00002A9794800F0B8FD784D794EDFF8E48117
:1030E00048B1822028602220794630608220C8F8CA
:1030F0000010BDE8FE839DF80800800701D4FFF7AB
:10310000BFFE02208DF80000200C8DF80100200A7F
:103110008DF802008DF803408DF8047000BF00BFE9
:1031200000BF00BF00BF00BF00BF00BF00BF00BFA7
:1031300000BF00BF00BF00BF00BF00BF00BF00BF97
:1031400000BF00BF00BF00BF00BF00BF00BF00BF87
:1031500000BF00BF00BF00BF00BF00BF4024554FED
:10316000FC6105216846FFF7B8F9BC6100BF00BFEC
:1031700000BF00BF00BF00BF00BF00BF00BF00BF57
:1031800000BF00BF00BF00BF00BF00BF00BF00BF47
:1031900000BF00BF00BF00BF00BF00BF00BF00BF37
:1031A00000BF00BF00BF00BF00BF00BF00202860FD
:1031B00079463060C8F800109BE72DE9FC5F3F4D71
:1031C0003F4E404F5FEA020A8B4604464FF000082C
:1031D0000DD001A9384800F037FD80B18220286069
:1031E00021203060784638608220BDE8FC9FC5F819
:1031F00000807846C6F8008038600020F5E703209C
:103200008DF80000200C8DF80100200A8DF80200D6
:103210008DF8034000BF00BF00BF00BF00BF00BF6C
:1032200000BF00BF00BF00BF00BF00BF00BF00BFA6
:1032300000BF00BF00BF00BF00BF00BF00BF00BF96
:1032400000BF00BF00BF00BF00BF00BF00BF00BF86
:1032500000BF00BF174C4FF04009C4F81C90042178
:103260006846FFF73AF951465846FFF742F9C4F865
:10327000189000BF00BF00BF00BF00BF00BF00BF6D
:1032800000BF00BF00BF00BF00BF00BF00BF00BF46
:1032900000BF00BF00BF00BF00BF00BF00BF00BF36
:1032A00000BF00BF00BF00BF00BF00BF00BF00BF26
:1032B00000BF9CE700800920A0860100800000106C
:1032C00084000010880000102DE9F05FFE4EDFF84A
:1032D000FC93DFF8FCA3150083460F464FF000086F
:1032E0000ED000240AE0395D0BEB0400FFF7ECFE82
:1032F000000602D53068BDE8F09F641CAC42F2D3F2
:10330000C6F800807946C9F800800020CAF800108D
:10331000F1E72DE9FC47044601A9EE4800F094FCD2
:10332000E94DEA4EDFF8A89348B1822028602220B8
:10333000794630608220C9F80010BDE8FC879DF80E
:103340000400800701D4FFF79BFD20208DF80000CA
:1033500020098DF8010020018DF8020000248DF86D
:10336000034000BF00BF00BF00BF00BF00BF00BFE1
:1033700000BF00BF00BF00BF00BF00BF00BF00BF55
:1033800000BF00BF00BF00BF00BF00BF00BF00BF45
:1033900000BF00BF00BF00BF00BF00BF00BF00BF35
:1033A00000BF4027DFF83083C8F81C70042168464E
:1033B000FFF793F8C8F8187000BF00BF00BF00BF48
:1033C00000BF00BF00BF00BF00BF00BF00BF00BF05
:1033D00000BF00BF00BF00BF00BF00BF00BF00BFF5
:1033E00000BF00BF00BF00BF00BF00BF00BF00BFE5
:1033F00000BF00BF00BF00BF2C60794634600020D2
:10340000C9F8001099E72DE9FC478A46044601A94E
:10341000B04800F019FCAC4DAC4EDFF8B49240B1AE
:10342000822028602220794630608220C9F800106E
:1034300083E703208DF8000020098DF801002001AA
:103440008DF8020000248DF8034000BF00BF00BFCC
:1034500000BF00BF00BF00BF00BF00BF00BF00BF74
:1034600000BF00BF00BF00BF00BF00BF00BF00BF64
:1034700000BF00BF00BF00BF00BF00BF00BF00BF54
:1034800000BF00BF00BF00BF00BF4027DFF8488279
:10349000C8F81C7004216846FFF71FF8B9015046B0
:1034A000FFF727F8C8F8187000BF00BF00BF00BFC3
:1034B00000BF00BF00BF00BF00BF00BF00BF00BF14
:1034C00000BF00BF00BF00BF00BF00BF00BF00BF04
:1034D00000BF00BF00BF00BF00BF00BF00BF00BFF4
:1034E00000BF00BF00BF00BF2C60794634600020E1
:1034F000C9F8001021E72DE9F34F83B0044601A974
:10350000744800F0A1FB704D704E714F4FF082086F
:1035100018B12120C5F800806CE09DF804008007F8
:1035200001D4FFF7ADFCAD208DF8000020098DF827
:10353000010020018DF802004FF0000B8DF803B060
:1035400000BF00BF00BF00BF00BF00BF00BF00BF83
:1035500000BF00BF00BF00BF00BF00BF00BF00BF73
:1035600000BF00BF00BF00BF00BF00BF00BF00BF63
:1035700000BF00BF00BF00BF00BF00BF00BF00BF53
:10358000DFF854914FF0400A5446C9F81CA00421BA
:103590006846FEF7A2FF02210498FEF79EFFC9F8D5
:1035A000184000BF00BF00BF00BF00BF00BF00BF8A
:1035B00000BF00BF00BF00BF00BF00BF00BF00BF13
:1035C00000BF00BF00BF00BF00BF00BF00BF00BF03
:1035D00000BF00BF00BF00BF00BF00BF00BF00BFF3
:1035E00000BF022401A93B4800F02EFB48B1222075
:1035F000C5F80080306078463860822005B0BDE8AC
:10360000F08F00BF00BF00BF00BF00BF00BF00BF02
:1036100000BF00BF00BF00BF00BF00BF00BF00BFB2
:1036200000BF00BF00BF00BF00BF00BF00BF00BFA2
:1036300000BF00BF00BF00BF00BF00BF00BF00BF92
:1036400000BFC9F81CA0AD20FEF740FF049802217E
:103650002044FEF742FFC9F818A000BF00BF00BF1A
:1036600000BF00BF00BF00BF00BF00BF00BF00BF62
:1036700000BF00BF00BF00BF00BF00BF00BF00BF52
:1036800000BF00BF00BF00BF00BF00BF00BF00BF42
:1036900000BF00BF00BF00BF00BFA41CA4B2B4F5B0
:1036A000805F9FD301A90B4800F0CEFA00287FF479
:1036B00030AFFFF72EFCC5F800B07846C6F800B072
:1036C000386000209AE7000080000010840000109D
:1036D00088000010A08601000080092070B5FD4D13
:1036E000FD4EFE4C2AB1FFF768FD000609D52068A3
:1036F00070BD8620206009202860784630608620D2
:1037000070BD00202060286078463060002070BDC9
:103710002DE9F04F89B0DFF8C483DFF8B8B35FEA72
:1037200002094FF0000607910FD04FF48055014673
:103730002A466846FCF7D1FDDDE90047284601F03E
:10374000C7F85FEA000A0CD016E08621C8F800101E
:103750000921CBF800107946DF480160862009B0C6
:103760004DE78221C8F800102221CBF800107946DD
:10377000D94801608220F2E7A9EB0605C7F5805021
:10378000A84200D20546B5F5805F04D020465146D8
:10379000FFF739FE80B92046FFF7BBFD60B90798F7
:1037A0002A46811907EB0A00FCF702FE2E44204648
:1037B0005146FFF7A0FE28B1504601F061F8D8F855
:1037C0000000CCE70027641C4E45D5D3504601F0DD
:1037D00057F80020C8F800007946CBF80000BE4832
:1037E00001600020BBE72DE9FF4F8DB00D46DDF8ED
:1037F00068900026B94C07935FEA09013FD04FF467
:10380000805701463A466846FCF767FDDDE900B19E
:103810000C913A46691C6846FCF75FFDDDE9001033
:10382000CDE904013A4668460F99FCF756FDDDE9FB
:10383000008500BFA9EB0607C5F58050B84200D24D
:10384000074625B1D8457CD10C98854279D14FF4F3
:10385000805001F03DF85FEA000A1BD0D8454FD1F7
:103860000C9885424CD12A464FEA08305146FFF762
:10387000A4FC000618D5504601F002F879E0862035
:1038800020609448092101607846934908608620A9
:1038900011B0B4E6822020608E4822210160794672
:1038A0008D4801608220F3E70598804509D104998D
:1038B00001EB0030C1F580525144FFF77EFC000659
:1038C000D9D44046FFF725FD0006D4D407983A46E0
:1038D000811905EB0A00FCF76BFDEA194FEA083085
:1038E0005146FFF7F1FC0006C5D40599884533D150
:1038F000049800EB01300499C1F58052514427E04F
:10390000059988450AD1049800EB01300499C1F566
:1039100080525146FFF751FC0006ACD44046FFF7F9
:10392000F8FC0006A7D407983A4681190F9830444E
:10393000FFF7CAFC00069ED4059988450CD104986F
:1039400000E00DE000EB01300499C1F580525146D2
:10395000FFF7BAFC00068ED4504600F091FF0AE053
:1039600007983A4681190F983044FFF7ADFC0006DE
:1039700001D520688CE73E44002508F101084E453A
:10398000FFF458AF53490020206008607846524940
:10399000086000207CE72DE9F0474FF0000900BFE8
:1039A00000BF00BF00BF00BF00BF00BF00BF00BF1F
:1039B00000BF00BF00BF00BF00BF00BF00BF00BF0F
:1039C00000BF00BF00BF00BF00BF00BF00BF00BFFF
:1039D00000BF00BF00BF00BF00BF00BF00BF402549
:1039E0003F4EF5619F20FEF771FD0020FEF76EFD52
:1039F00000F0FF080020FEF769FDC4B20020FEF7CA
:103A000065FDC1B2B56100BF00BF00BF00BF00BF10
:103A100000BF00BF00BF00BF00BF00BF00BF00BFAE
:103A200000BF00BF00BF00BF00BF00BF00BF00BF9E
:103A300000BF00BF00BF00BF00BF00BF00BF00BF8E
:103A400000BF00BF00BF254D224E234FB8F1BF0F6E
:103A500003D1252C0AD0262C08D0822028602120D2
:103A60003060784638608220BDE8F0871D484129E3
:103A700012D04FF48002422912D04A2910D0C0F847
:103A800000900020FFF78EFAC5F800907846C6F83F
:103A9000009038600020E7E74FF400110160F0E784
:103AA0000260EEE72DE9F84F69460F4800F0CCF8C8
:103AB00082270A4C074D084E4FF0220A002862D197
:103AC0009DF80000800701D4FFF7DAF900BF00BFBE
:103AD00000BF0BE084000010880000108000001080
:103AE0000080092028010010A086010000BF00BF4F
:103AF00000BF00BF00BF00BF00BF00BF00BF00BFCE
:103B000000BF00BF00BF00BF00BF00BF00BF00BFBD
:103B100000BF00BF00BF00BF00BF00BF00BF00BFAD
:103B200000BF00BF00BFDFF8EC914FF04008C9F8BC
:103B30001C806020FEF7CAFCC9F8188000BF00BFD7
:103B400000BF00BF00BF00BF00BF00BF00BF00BF7D
:103B500000BF00BF00BF00BF00BF00BF00BF00BF6D
:103B600000BF00BF00BF00BF00BF00BF00BF00BF5D
:103B700000BF00BF00BF00BF00BF00BF694666486E
:103B800000F062F838B127607846C5F800A03060D0
:103B90008220BDE8F88F00202060286078463060E1
:103BA0000020F6E75D48006870474FF4805070478A
:103BB0002DE9F04FDFF86881DFF868B189B00F00B8
:103BC00004464FF0000626D04FF4805501462A46A1
:103BD0006846FCF782FBDDE900A105912A462146F3
:103BE00006A8FCF77AFBDDE906404FF00009BD1B93
:103BF000C0F58051A94200D20D4620B1544515D1DF
:103C00000599884212D12046FFF783FB00060DD5A7
:103C1000D8F80000A3E58621C8F800100921CBF8E8
:103C20000010794640480160862098E52E44641CC7
:103C30004846BE42DBD3C8F800007946CBF8000006
:103C40003948016000208AE52DE9F041374C0F46E4
:103C50000646A56806E0A068401BB04202D30120DA
:103C6000BDE8F081384600F003F80028F3D1F7E70B
:103C700070B5044600BF00BF00BF00BF00BF00BF5B
:103C800000BF00BF00BF00BF00BF00BF00BF00BF3C
:103C900000BF00BF00BF00BF00BF00BF00BF00BF2C
:103CA00000BF00BF00BF00BF00BF00BF00BF00BF1C
:103CB00000BF00BF4025174EF5610520FEF706FC4A
:103CC0000020FEF703FC2070B56100BF00BF00BFFD
:103CD00000BF00BF00BF00BF00BF00BF00BF00BFEC
:103CE00000BF00BF00BF00BF00BF00BF00BF00BFDC
:103CF00000BF00BF00BF00BF00BF00BF00BF00BFCC
:103D000000BF00BF00BF00BF00BF207800F001006F
:103D100070BD00000080092020A1070028010010CC
:103D2000800000108400001088000010000009408E
:103D30002DE9FF4703A9FE4800F05FFBFD4DFE4E55
:103D4000DFF8F89350B18220286021207946306056
:103D50008220C9F8001004B0BDE8F0879DF80C007F
:103D6000800701D4FFF78CF842208DF80000002472
:103D7000CDF80140CDF80540ADF8094000BF00BFC7
:103D800000BF00BF00BF00BF00BF00BF00BF00BF3B
:103D900000BF00BF00BF00BF00BF00BF00BF00BF2B
:103DA00000BF00BF00BF00BF00BF00BF00BF00BF1B
:103DB00000BF00BF00BF00BF00BF00BF4027DFF84B
:103DC0008083C8F81C700B216846FEF786FBC8F894
:103DD000187000BF00BF00BF00BF00BF00BF00BF22
:103DE00000BF00BF00BF00BF00BF00BF00BF00BFDB
:103DF00000BF00BF00BF00BF00BF00BF00BF00BFCB
:103E000000BF00BF00BF00BF00BF00BF00BF00BFBA
:103E100000BF2C60794634600020C9F800109AE792
:103E20002DE9F34F85B0044603A9C14800F0E5FA37
:103E3000C04DC14EC14F4FF0820B18B12120C5F8C3
:103E400000B060E0FFF71CF842208DF800004FF052
:103E5000000ACDF801A0CDF805A0ADF809A000BF7B
:103E600000BF00BF00BF00BF00BF00BF00BF00BF5A
:103E700000BF00BF00BF00BF00BF00BF00BF00BF4A
:103E800000BF00BF00BF00BF00BF00BF00BF00BF3A
:103E900000BF00BF00BF00BF00BF00BF00BFDFF812
:103EA000A0924FF04008C9F81C800B216846FEF72D
:103EB00014FBC9F8188000BF00BF00BF00BF00BFDF
:103EC00000BF00BF00BF00BF00BF00BF00BF00BFFA
:103ED00000BF00BF00BF00BF00BF00BF00BF00BFEA
:103EE00000BF00BF00BF00BF00BF00BF00BF00BFDA
:103EF00000BF00BF00BF03A98D4800F07EFA48B1A3
:103F00002220C5F800B0306078463860822007B0C3
:103F1000BDE8F08F9DF80C00800701D4FEF7B0FFDC
:103F200002208DF80000200C8DF80100200A8DF889
:103F3000020006988DF803408DF8040000BF00BF12
:103F400000BF00BF00BF00BF00BF00BF00BF00BF79
:103F500000BF00BF00BF00BF00BF00BF00BF00BF69
:103F600000BF00BF00BF00BF00BF00BF00BF00BF59
:103F700000BF00BF00BF00BF00BF00BF4446C8462F
:103F8000C9F81C4005216846FEF7A7FAC8F8184092
:103F900000BF00BF00BF00BF00BF00BF00BF00BF29
:103FA00000BF00BF00BF00BF00BF00BF00BF00BF19
:103FB00000BF00BF00BF00BF00BF00BF00BF00BF09
:103FC00000BF00BF00BF00BF00BF00BF00BF00BFF9
:103FD000C5F800A07846C6F800A03860002096E733
:103FE0002DE9F05F534EDFF85091DFF850A1150036
:103FF00083460F464FF000080ED000240AE0395DDA
:104000000BEB0400FFF70CFF000602D53068BDE89B
:10401000F09F641CAC42F2D3C6F800807946C9F820
:1040200000800020CAF80010F1E72DE9F34F0024CA
:10403000404D414E414FC3B080464FF0820A4FF091
:10404000210BA14641A93A4800F0D7F900286ED1CA
:104050009DF80401800701D4FEF712FF02208DF8BD
:1040600000004FEA18108DF8010004EB08108DF8DD
:10407000020044988DF8039000EB04214FF4807205
:1040800001A8FCF795F900BF00BF00BF00BF00BF4B
:1040900000BF00BF00BF00BF00BF00BF00BF00BF28
:1040A00000BF00BF00BF00BF00BF00BF00BF00BF18
:1040B00000BF00BF00BF00BF00BF00BF00BF00BF08
:1040C00000BF00BF00BF40201D49C8614FF482718E
:1040D0006846FEF702FA1A494020886100BF00BF17
:1040E00000BF00BF00BF00BF00BF00BF00BF00BFD8
:1040F00000BF00BF00BF00BF00BF00BF00BF00BFC8
:1041000000BF00BF00BF00BF00BF00BF00BF00BFB7
:1041100000BF00BF00BF00BF00BF00BF641CE4B20F
:10412000102C8FD341A9024800F067F998B109E03B
:10413000A08601008000001084000010880000109C
:1041400000800920C5F800A07846C6F800B03860A5
:10415000822045B0DCE6FEF7DCFEC5F8009078462C
:10416000C6F8009038600020F3E72DE9F04F89B0E1
:10417000DFF85083DFF850B35FEA02094FF0000622
:1041800007910FD04FF4805501462A466846FCF748
:10419000A4F8DDE90047284600F09AFB5FEA000A30
:1041A0000CD016E08621C8F800100921CBF80010C9
:1041B0007946C6480160862009B0A9E68221C8F880
:1041C00000102221CBF800107946C04801608220FF
:1041D000F2E7A9EB0605C7F58050A84200D20546D4
:1041E000B5F5805F04D020465146FFF70CF980B941
:1041F0002046FFF78EF860B907982A46811907EB29
:104200000A00FCF7D5F82E4420465146FFF70DFF73
:1042100028B1504600F034FBD8F80000CCE7002766
:10422000641C4E45D5D3504600F02AFB0020C8F848
:1042300000007946CBF80000A44801600020BBE7ED
:104240002DE9FF4F8DB00D46DDF8689000269D4C9E
:1042500007935FEA09013ED04FF4805701463A4682
:104260006846FCF73AF8DDE900B10C913A46691C62
:104270006846FCF732F8DDE90010CDE904013A4662
:1042800068460F99FCF729F8DDE90085A9EB0607D8
:10429000C5F58050B84200D2074625B1D8457CD13B
:1042A0000C98854279D14FF4805000F011FB5FEA01
:1042B000000A1BD0D8454FD10C9885424CD12A46D4
:1042C0004FEA08305146FEF778FF000618D55046F1
:1042D00000F0D6FA79E0862020607B480921016051
:1042E00078467A490860862011B011E68220206065
:1042F0007548222101607946744801608220F3E705
:104300000598804509D1049901EB0030C1F5805230
:104310005144FEF752FF0006D9D44046FEF7F9FF9C
:104320000006D4D407983A46811905EB0A00FCF739
:104330003FF8EA194FEA08305146FFF751FE0006F0
:10434000C5D40599884533D1049800EB0130049910
:10435000C1F58052514427E0059988450AD1049857
:1043600000EB01300499C1F580525146FEF725FF5C
:104370000006ACD44046FEF7CCFF0006A7D4079851
:104380003A4681190F983044FFF72AFE00069ED462
:10439000059988450CD1049800E00DE000EB013050
:1043A0000499C1F580525146FFF71AFE00068ED4DB
:1043B000504600F065FA0AE007983A4681190F98CE
:1043C0003044FFF70DFE000601D520688CE73E441F
:1043D000002508F101084E45FFF458AF3A49002086
:1043E0002060086078463949086000207CE74FF477
:1043F000800070474FF4805070472DE9F041344CF5
:104400000F460646A56806E0A068401BB04202D3EE
:104410000120BDE8F081384600F003F80028F3D110
:10442000F7E770B5044600BF00BF00BF00BF00BF84
:1044300000BF00BF00BF00BF00BF00BF00BF00BF84
:1044400000BF00BF00BF00BF00BF00BF00BF00BF74
:1044500000BF00BF00BF00BF00BF00BF00BF00BF64
:1044600000BF00BF00BF40251A4EF5610520FEF7D2
:104470002DF80020FEF72AF82070B56100BF00BFBC
:1044800000BF00BF00BF00BF00BF00BF00BF00BF34
:1044900000BF00BF00BF00BF00BF00BF00BF00BF24
:1044A00000BF00BF00BF00BF00BF00BF00BF00BF14
:1044B00000BF00BF00BF00BF00BF00BF207800F0FA
:1044C000010070BD80000010840000108800001002
:1044D000000009400080092000207047AE4982207A
:1044E0000860AE49212008607846AD490860822006
:1044F0007047A94982200860A849222008607846B0
:10450000A749086082207047A34982200860A34918
:10451000222008607846A24908608220704770B562
:10452000002400BF00BF00BF00BF00BF00BF00BF2E
:1045300000BF00BF00BF00BF00BF00BF00BF00BF83
:1045400000BF00BF00BF00BF00BF00BF00BF00BF73
:1045500000BF00BF00BF00BF00BF00BF00BF00BF63
:1045600000BF40258F4EF5619F20FDF7AFFF002073
:10457000FDF7ACFF60F307040020FDF7A7FF60F331
:104580000F240020FDF7A2FF60F31744B56100BFC0
:1045900000BF00BF00BF00BF00BF00BF00BF00BF23
:1045A00000BF00BF00BF00BF00BF00BF00BF00BF13
:1045B00000BF00BF00BF00BF00BF00BF00BF00BF03
:1045C00000BF00BF00BF00BF00BF00BF00BF7649F3
:1045D000601A8C421AD00BDCA4F1C204B4F5A11409
:1045E00014D0B4F5803F11D0B4F5003F0BD10DE0ED
:1045F0006E49401805D06E49401809D06D49C8422F
:1046000001D1022400E00024204670BD0324FBE712
:104610000424FFF78DFBF7E76748007828B1674966
:1046200000EBC00051F8200000475B498220086081
:104630005A4921200860784659490860822070470D
:1046400070B5FFF76CFF5C49544D554E524C0870E5
:1046500050B15A4900EBC00001EB800080688047F0
:10466000000609D5206870BD8220206021202860C6
:1046700078463060822070BD002020602860784637
:104680003060002070BD2DE9F0414B4B434D444E4E
:104690001B78414C63B19AB1484F03EBC30307EB5E
:1046A00083031B699847000612D52068BDE8F08196
:1046B0008220206021202860784630608220F5E743
:1046C0008620206009202860784630608620EDE74B
:1046D000002020602860784630600020E6E72DE961
:1046E000F041354B2D4D2E4E1B782B4C5BB192B1CA
:1046F000324F03EBC30307EB83039B699847000624
:1047000011D52068D2E782202060222028607846D8
:1047100030608220CAE78620206009202860784621
:1047200030608620C2E70020206028607846306034
:104730000020BBE7F8B5204C184D194E2778164CD1
:10474000DDF818C087B1BCF1000F15D0CDF800C05E
:10475000DFF868C007EBC7070CEB8707FF69B847AE
:10476000000611D52068F8BD822020602220286034
:10477000784630608220F8BD8620206009202860BD
:10478000784630608620F8BD00202060286078469A
:1047900030600020F8BD0000800000108400001090
:1047A0008800001000800920C220180003FBD6FFFB
:1047B00000FFFEFF0001F8FF2C010010504F000029
:1047C00070B500242546002801DA01244042002962
:1047D00001DA0125494200F019F8AC4200D040420C
:1047E000002C00D0494270BD064C074D06E0E06841
:1047F00040F0010394E8070098471034AC42F6D328
:10480000FBF774FC285000004850000030B50B4600
:10481000014600202022012409E021FA02F59D42F0
:1048200005D303FA02F5491B04FA02F52844151EC4
:10483000A2F10102F1DC30BD30B58C1810F8012B6B
:1048400012F00F0301D110F8013B120906D110F844
:10485000012B03E010F8015B01F8015B5B1EF9D14D
:1048600001E001F8013B521EFBD1A142E6D300203A
:1048700030BD002001E001C1121F002AFBD17047AA
:1048800010B5002821D0114B0022001F196803E049
:10489000814203D80A4649680029F9D152B1136808
:1048A000841A9C4204D1006818441060104602E04B
:1048B000506000E0186039B102680B1A934203D1CE
:1048C0000B681A4402604968416010BD3001001055
:1048D000F0B50B30154D20F007010024144A0FE00D
:1048E00003688B420BD38B4205D95E1A4318476885
:1048F000C3E9006700E04368136002C004E0021DE2
:1049000010680028ECD12046002802D1286808B1A0
:104910000020F0BD064A07481060074A121A22F02C
:104920000702C0E9002401202860D7E73401001005
:10493000300100107C1D0010788D001000050F0A5A
:104940001B1E141133363C39282D272263666C69EF
:10495000787D777250555F5A4B4E4441C3C6CCC9DF
:10496000D8DDD7D2F0F5FFFAEBEEE4E1A0A5AFAACF
:10497000BBBEB4B193969C99888D878283868C89BF
:10498000989D9792B0B5BFBAABAEA4A1E0E5EFEAAF
:10499000FBFEF4F1D3D6DCD9C8CDC7C240454F4A9F
:1049A0005B5E545173767C79686D676223262C298F
:1049B000383D373210151F1A0B0E040103060C097F
:1049C000181D171230353F3A2B2E242160656F6A6F
:1049D0007B7E747153565C59484D4742C0C5CFCA5F
:1049E000DBDED4D1F3F6FCF9E8EDE7E2A3A6ACA94F
:1049F000B8BDB7B290959F9A8B8E848180858F8A3F
:104A00009B9E9491B3B6BCB9A8ADA7A2E3E6ECE92E
:104A1000F8FDF7F2D0D5DFDACBCEC4C143464C491E
:104A2000585D575270757F7A6B6E646120252F2A0E
:104A30003B3E343113161C19080D070200002110EB
:104A4000422063308440A550C660E77008812991F8
:104A50004AA16BB18CC1ADD1CEE1EFF131121002A0
:104A600073325222B5529442F772D6623993188348
:104A70007BB35AA3BDD39CC3FFF3DEE3622443346C
:104A800020040114E664C774A44485546AA54BB598
:104A900028850995EEE5CFF5ACC58DD55336722640
:104AA00011163006D776F6669556B4465BB77AA7E8
:104AB00019973887DFF7FEE79DD7BCC7C448E5588C
:104AC0008668A7784008611802282338CCC9EDD938
:104AD0008EE9AFF9488969990AA92BB9F55AD44AE0
:104AE000B77A966A711A500A333A122AFDDBDCCB88
:104AF000BFFB9EEB799B588B3BBB1AABA66C877CAC
:104B0000E44CC55C222C033C600C411CAEED8FFDD7
:104B1000ECCDCDDD2AAD0BBD688D499D977EB66E7F
:104B2000D55EF44E133E322E511E700E9FFFBEEF27
:104B3000DDDFFCCF1BBF3AAF599F788F8891A981E9
:104B4000CAB1EBA10CD12DC14EF16FE18010A100D3
:104B5000C230E3200450254046706760B9839893C3
:104B6000FBA3DAB33DC31CD37FE35EF3B102901223
:104B7000F322D2323542145277625672EAB5CBA58F
:104B8000A89589856EF54FE52CD50DC5E234C32473
:104B9000A01481046674476424540544DBA7FAB763
:104BA0009987B8975FE77EF71DC73CD7D326F236C3
:104BB0009106B01657667676154634564CD96DC9AF
:104BC0000EF92FE9C899E9898AB9ABA94458654813
:104BD00006782768C018E1088238A3287DCB5CDB03
:104BE0003FEB1EFBF98BD89BBBAB9ABB754A545A63
:104BF000376A167AF10AD01AB32A923A2EFD0FEDCF
:104C00006CDD4DCDAABD8BADE89DC98D267C076CB2
:104C1000645C454CA23C832CE01CC10C1FEF3EFFA2
:104C20005DCF7CDF9BAFBABFD98FF89F176E367E02
:104C3000554E745E932EB23ED10EF01E005EBCE265
:104C4000613FDD83C29C7E20A3FD1F419DC3217F68
:104C5000FCA2401E5F01E3BD3E6082DC237D9FC15C
:104C6000421CFEA0E1BF5D0380DE3C62BEE0025C50
:104C7000DF81633D7C22C09E1D43A1FF4618FAA43C
:104C800027799BC584DA3866E5BB5907DB85673928
:104C9000BAE406581947A5FB7826C49A653BD9871C
:104CA000045AB8E6A7F91B45C6987A24F8A6441A10
:104CB00099C7257B3A6486D85B05E7B98CD2306EFC
:104CC000EDB3510F4E10F2AC2F7193CD114FADF3E8
:104CD000702ECC92D38D6F31B2EC0E50AFF1134DDC
:104CE000CE90722C6D33D18F0C52B0EE326C8ED0D0
:104CF000530DEFB1F0AE4C1291CF2D73CA947628BC
:104D0000ABF517490856B4EA6937D58B5709EBB5A7
:104D100036688AD495CB2977F4AA4816E9B7550B9B
:104D200088D6346A2B7597C94A14F6A8742AC8968F
:104D3000154BA9F7B6E80A54D7896B35EB3C904D73
:104D400053444F53352E3000020201000110000081
:104D500004F80C0001000100000000000000000049
:104D6000000029EFBEADDE41544F4C204650726921
:104D70006E744641543132202020000000000000B3
:104D80000010000000200000003000000040000083
:104D90000050000000600000007000000080000073
:104DA0000090000000A0000000B0000000C0000063
:104DB00000D0000000E0000000F000000000010052
:104DC00000800100000002000080020000000300DB
:104DD00000800300000004000080040000000500C3
:104DE00000800500000006000080060000000700AB
:104DF00000800700FF0F0000FF1F0000FF2F0000D2
:104E0000FF3F0000FF4F0000FF5F0000FF6F00004A
:104E1000FF7F0000FF8F0000FF9F0000FFAF00003A
:104E2000FFBF0000FFCF0000FFDF0000FFEF00002A
:104E3000FFFF0000FF7F0100FFFF0100FF7F020076
:104E4000FFFF0200FF7F0300FFFF0300FF7F04005E
:104E5000FFFF0400FF7F0500FFFF0500FF7F060046
:104E6000FFFF0600FF7F0700FFFF07001201100190
:104E70000000004051C20313000104204801090250
:104E8000200001010080320904000002080650627F
:104E900007058202400000070502024000000004EE
:104EA0000309041C03410054004F004C0020002063
:104EB00000200020002000200020002000200028EA
:104EC0000346005000720069006E00740020004626
:104ED000006C0061007300680020002000200020AA
:104EE000002000200020001A034600690072006DB7
:104EF0000077006100720065003000300030003043
:104F0000000E034D0065006D006F00720079000017
:104F1000FD1E0000000000007F24000000000000D3
:104F20000000000000000000000000000000000081
:104F30000000000000000000000000000000000071
:104F40000000000000000000000000000000000061
:104F5000D9440000D9440000DD440000F3440000BF
:104F6000DD440000F3440000F3440000F34400007B
:104F700009450000D9440000D9440000DD44000088
:104F8000F3440000DD440000F3440000F34400005B
:104F9000F344000009450000A53B0000AB3B0000C6
:104FA00097390000A53A0000DD36000011370000F7
:104FB000C9320000E7370000B13B0000EB2C0000D5
:104FC000F12C0000F5270000A53A0000DD360000B6
:104FD000492A0000E13F00003D2B0000F72C0000B3
:104FE000EF430000F543000097390000A53A0000A8
:104FF000DD3600006B410000E13F0000414200004F
:10500000B13B0000000000000000000000000000B4
:105010000000000000000000000000000000000090
:1050200000000000000000004850000000000010D8
:1050300038010000384800007450000038010010AA
:10504000409C0000724800000114BD41544F4C20A8
:10505000465072696E74280548D4284B3D321302BD
:1050600066102C0E270780C3C90100879303044DE7
:105070006CDC0200CFB05F8019902B6387DCEDB54C
:1050800086DA631A49E3F642CCCF19D1A890DE82C2
:10509000D1093EC932A0B1026D132C443F6FE20B1F
:1050A0005DC29A8FDD3A8604A0CFE9F04291BC9FA1
:1050B000A90D391B343AC1B862C004895FEE93ABC5
:1050C00044BF2AFA92F55DBDC0E5E8254FB8C52773
:1050D000BE7839E59573278AC6BD439D6E516F67CB
:1050E000DCE852A7875BA2CFA751834BA9E47C0FD2
:1050F0006DABC74CCCA3DB283EA4A5C20EA3FA0916
:10510000B5D3BCDBE638D196C25AD8E4AB939B1832
:105110000ED7BF38788BC204469F315C40EE8FC5F6
:1051200046CCFF9FFFD51D01AD9E2C5DD2AB1B4031
:1051300093876C18EC2957D76B5B8777D865D5BCFC
:10514000E535824D2DBCD2F9B634151D34B38F77B9
:10515000C972956992599FD31CE6F879B848DA2B41
:1051600020E74BEFD35B76461A93A7EF593539F416
:105170008881A38F587365E2E0678D7AC78F27A176
:105180005AF357F406755CAFBDBAA2005849FF2D1B
:10519000ED8D671E983FD1C609C24CE9877DC320BB
:1051A000B2EC9ADF10969820D45BBE14AAD7F6DA38
:1051B000CA5913325DA15EC04CA26A123C27A0D727
:1051C00042CDCF97A9F166B749FD0E2990A934DFEA
:1051D00051C13EE2337FBA97D609AD226D9F8E480A
:1051E0008FEE0E376CB191C0F5CA386395F5ACAD52
:1051F000DB511784F8F5683D180473D5E48A756EA1
:10520000C46E451AB2ED333679B0BD1C4DB48EC8AC
:105210008EAE31D971D2D1822EF17FE225EFB48AE0
:1052200029574B5EFE53332DEC2EC347B6BE775F36
:105230003280B01214C3036ECE09AEC9CDB6287F3A
:10524000044BD8215D6C482873AD930FE70500022D
:10525000765F8DB0F3FF5D72B5A76D8A333727ECAB
:105260007D52528FBFB2C11DA2A1FF15967C3A9705
:105270006EBF8CE3399B658AF1810FBB8B38F1508F
:105280004AD90669E582B61FDA7834E664607CBEE6
:10529000D210922F0772C3CCF21F9E8B91DF6A123D
:1052A0009DB7858214A567B6ED78C5DEEE51F6F799
:1052B00041A0D0D9C5DD261F72E23049384E444E98
:1052C0004E77472E5F94B73AC9683FDD1678D4AC65
:1052D000FF4605109D8FCC13375C9C6B87E70B1E38
:1052E00050093E3496CF07364D72F34D6056D7C9FC
:1052F000BF0D1193123197E19A22F403D137BB729B
:105300001429EA945DC3273E625120DFB48514213D
:10531000F1E12B321121477A83E76BDFDB3D313935
:105320002CC034BE0E3ABC1B8A138621B1C7965BD3
:10533000D9AE8CD928F16C90EF2CC285E29375C15F
:105340008BE21C4D84B06A70AB8CDD2A6BB31D857B
:1053500055826E8109E158E305EF75B1423CA84BD7
:105360007AEAA6155C982675ABB569691077BD0613
:10537000BDD46EF72D6E69F6FD1D70B468F644F06D
:1053800063F1AF189DCFF3F3EF312A55A1FAC0D1E5
:10539000888716EFDD3D51E67BA968EA6131783DEB
:1053A000D047B7BC032F6EAD84B4F9BF23AD4C0515
:1053B0004DAFFD4831402EAC21BDC6DE1CFD57F07F
:1053C000ADD62497EA030AFA5D5DAE6510934514E5
:1053D000CA6F8632D4E745532FD08B2855D2B9985F
:1053E000AC1C7A6C2CB6E7C7056F7D52E9E8CD9608
:1053F0001BFC1427298827BE6AACB5794DB0235D04
:10540000E00397EC2309255114E84F294BF0E2B74C
:105410004CF894A405420C0BCEBFB664A39043F5A0
:10542000FEC47935B092B9C7E18A1BA9664373D22D
:105430000454A0AA478AFCB050127A36B224AD09AF
:105440003B1A6B2C95B3EE28F2A7541A6A6183F5C8
:10545000B8099017C39B2DA08645C217961A30999C
:10546000A2B9561F8319CC401E2E90C1116A12DCBE
:10547000CFC94889B78AD0AF3254E9F4353F868125
:10548000DE76753EC579345F0AC728638A8F0FC1FF
:1054900035142D3283F5BC8E299A216A038AFD16B4
:1054A000A47007E56EE5F5021740B44FBAEA277716
:1054B000756D889CAE87FA716F356E9591BFD81F58
:1054C000BD5AB1A84CA5C231A843F3928A692CA257
:1054D000D5A229531FB22B79195A30E817BAF066B2
:1054E00045159BC8D397BC822611312DC7B0816565
:1054F0001D319F9D8F2D3CA31E64E2060BA2FA2A4C
:10550000F524E665A094D5C5A85E9686B0378B498C
:10551000B27884965349161C49E7AEAF0A8F0071E2
:105520003C6AA3CBAAD6BC71000FBBB4C78E319026
:1055300055B0D6D306041CBA56BDA19D7B9D7700FD
:10554000467676FAFFCEA44779102FE6CD15489D12
:1055500044BBEA115BBDEE0CFC108FB796D25CFA2F
:1055600058EDF75C40D73A5642AC0A038EC24E342F
:10557000ABF4AA8F73846C49AC5CFF0DF7B8EC5E9A
:10558000099D3FB8470A7F1B601879F1BE8760FB11
:105590006B9BE2760E5267687D8F7D3B5D7EDCE122
:1055A0007F3778864B3E0B8F6372548B8F169ED15C
:1055B00059712751A0ECCCED9481B21E85C7D57EE0
:1055C000CA2837C084BF3E06C1C7FAAA4D4C8A68B4
:1055D000C0D68BD543D72BB4376D569679EA2BDAE4
:1055E000262B49B66C6BB872D881A30FF8E30F99DC
:1055F00077B2D30C7944A247221679C459637A9CB6
:105600009BC203E0A80B110B0B39EA250F1DFF16F7
:10561000836F9128A30AA2E5BFC3F9BC3372179B1D
:105620002FEDEEF2598FBCFD8ECC2AD4EC1AE35646
:10563000EBAC190E938A2BA3796852E7EC5C09DB7B
:1056400085A206056A7076C0967CCA01A6469A8B2A
:10565000EB506AC35414717B40FAC8643B76308FB8
:105660009375F606F7CE04961A76B1CB7B078CB00D
:1056700058978D6E302F95EDEB1B57660FA090ACB1
:1056800046060466B931370C5AB0D89BCE8098B91B
:10569000CD27D026B55AD3055613FBFD4766F9E949
:1056A0003F8328971718E1A79DAB5A7F1910A0BD1B
:1056B000A8E248895EB6D5C1115F7EFE0570F30F82
:1056C000D034301CFC873F7F2B53B852996B650E4A
:1056D0008A7D6420E3B0E0D69CCC5B42AFD10A8DDA
:1056E000CBAEE2AB5FA23870036313B66B3EB2334E
:1056F0008012615B46F1C10CDC2B36BD66F3CF56E0
:10570000E2C1BB3B441001614CFE0FB2803F97F5F4
:10571000B077D4E0913F87140180E67D0A6F8FA2B5
:105720001BA5B4F167B4FBE3F797CD89545AE2E2C5
:10573000843D837623B61501667BC0FBC9AA8E1013
:10574000F19BBCF1C21FAC52AB152619A9920D15E5
:10575000270733C0F8D5B6E5BDA7F3A9AA7F5EEF4A
:1057600029ABC0DEC103A7FF42D177F782E4A9933A
:10577000E7EF4A6D7BA8660E219C1D1EF0DE7A2C99
:10578000AB2C0436F1D9383078B84F2616DA010838
:10579000E05CBA140881CBBED00ABBCE7937A79A99
:1057A00088F720E07C93717643ACD2DA0395454BC1
:1057B000E27F9E1F242C5C000D6591CA173FB56CDB
:1057C000EADAA48E77B35394F098BDF4C3684136F7
:1057D000FAF456C7796BB92591BDA8AA89BC7CBDDE
:1057E0004A0322CB3BD4051173A0989B17C0676A6C
:1057F0008C9323C0F36A74D8F48329353D52DBD0EF
:10580000C5B4CDD93524257444BFD03CD874B85024
:1058100029E832F25CBDD6D9C01F2110B691EDEC5B
:105820000D695CE0CA751FA71A6FF9FF5B8CBE6833
:105830002D2A5FE1F1FB43B50397657552FF1DF417
:10584000EC41B00C810C67B8D8C39A6230162402C0
:10585000D6A7CF18C150C463A58E96BDBC27BE3055
:105860005249CA30971750CE4A1D77DC5BC0D187AA
:105870001FBC602998366C407BA9F6310CE63537A1
:105880008B4CA687EB79EE3A182AAAA7323F52B67C
:10589000E8E6404003CCDD6B6F818B5A30A518637E
:1058A00055BE3721108F7E59A8B5B17960D36720D6
:1058B000952BBACAD4C87A4257F19ADFFCA44FE1BB
:1058C000EFAD137E58D893DF7705A4ABB24AA2C1DF
:1058D0000641A263E6E55B9893E6632D915F7A9FAC
:1058E00024684D98D1E2ADED600EC861C84F75BC1B
:1058F000ACEAD6AE2BB0B4D8A678E8D16E245E0858
:10590000D643CB1CA4EB3644B387212B60123E8FC9
:1059100060693C934FC79FF47878E98445FE9E4EBA
:10592000F8F58848A32FFE926F2C30FB909FF1373B
:10593000986DDFDBB3506181397AA5845125126FF0
:105940000BDAF89B2C9B11E60E28E2EA4E7BEAEC80
:10595000D974AFDC491C55F678FA692FCED4FF36DE
:105960008AF2FDAE8AAB167EF55BF2C0B18A3A547C
:105970001598FBAC827F54DA3E4E247692F5755032
:10598000B06E139DD6D6E237DCD1669EB4E6CF3337
:105990006ADF9329574F812E4CA55FF6A49EEEE94E
:1059A0006E3158D832A3B8E8CB4462D904D6E15D51
:1059B0004674BE23EA7E8F141A669666BF3377A4B8
:1059C000CA378C3E91FB062C470B4C853ABC4425CC
:1059D0003AD3F994F34958DA3AB37095D38CCD039E
:1059E0004A713B04CC7FB11E6014E9BA648E8D19F4
:1059F000BB6D7F0324B9B06A4D270244D035E1DE88
:105A00001F2335A49351A26145BC39B97E0928EA08
:105A1000109F5DB2F46DE9ECB6FBC7A19DFE73E685
:105A2000AE85949D89E15A4D589489E43BE925D08F
:105A3000ECD3D6F4FD1458F4863ED73F04A6C27AC0
:105A40009D90C4E0F73CC43E6D8323416DB3A72D08
:105A5000A56D7F2C423EC212B1D7DAFA00EB1B8152
:105A60000A3DDA1C3C1E6BB662B5139B4DDFABFEE4
:105A7000D7412606A595D0A6B6059D3FD5A2266599
:105A8000AB178C83B49D81C4C736D9E610A1741BB3
:105A9000BE32E7A181D1BA055FE91C229929FDF840
:105AA00056F6F289F2301BD93EE1C85B4AA39D76D7
:105AB00091C209CE076FD2081A2CC6591FD16B1B91
:105AC00070FE541852363B427D582DBDD1E1BE3395
:105AD00053B0D9A1763CE8007C7E9CB088529AD124
:105AE000384F1E4076565ACBCFA239E68ED2F029D7
:105AF000DD4A1734258319F520ACDAFFE986BA3B75
:105B0000DB514189FDBDBBD9D186EBEC9442DA4033
:105B10008866CD3D1B06B1559432F01FA7E5E4C859
:105B200070EE41F0BC232B4FB3E75D1F93E38F4032
:105B3000A9C0D6479A8138AC42C971723CB1187E6F
:105B4000AA51F7D0F5DDA17BD42F64F0F6C8859D6E
:105B5000A7A53F314B6E7D799A6F526C992CCDE29F
:105B60009067A9FE98CC94BF9B04C7AC8274EAEFFF
:105B700004DE619CD5B43A6437318D1B63B1AD64EA
:105B8000EDE32DDC744A099469614C744879A6539D
:105B90001A57E6FFBD3CD37610536A8A1CCD953B5D
:105BA000A15BDF4D0BDA7264398242358B2C015ACE
:105BB000EA24735CDF3825A2C94B51F1B740BEA976
:105BC000614E23E2405B77B48096AE2A7709851157
:105BD000A2FE08F1ACB1812711E1E1F8AFB5E076A2
:105BE0007570FBDC3923BA17756E41D9D82332277B
:105BF000F8BCB4AE39EE3CBA32D147782DFF689D7F
:105C0000AD1C606866855A5A0D2BDF35ED3968ACDE
:105C10006FD4B052DB385C2ACB82F8204FAD1442EF
:105C2000E548E163BFEC056DDDEDC2EB48CC5CF40B
:105C3000C70A4F773D3525016AFEE91BDB7B9CEDEA
:105C40008805A6C05E7233530174B1522163FAD144
:105C50001A44E9AF00D61C5E649A0F46D8C4B097C8
:105C6000A59B073ACA82879ECCC59E064C95A4D6B2
:105C7000061F75DAEFD41127674981ED55A8AA12DE
:105C8000B183AC1A2EAF50F517920AC9D8DB75CC88
:105C900041C3961B4BF36AC0F9A31FF13CA390923A
:105CA0007F7560DA73CE62B6241E2E749D83DD92FA
:105CB000298F0BBC621E40B8E2D9258DDECC1A704C
:105CC0007848BABB936F95B4842206D155EC792DF0
:105CD0001D1608F33698A4712A7999C0619290BF75
:105CE000490FD8F815DBCD65522525962AE9817034
:105CF0007E7497202434E5830A06528C0AE9180141
:105D0000528DC00A724C5ACC5BD9814C28ECB45BE2
:105D1000C8C4AFC5FE4D9F613BC44BACC33AAECCCB
:105D20005410AEB42C085E4479DF2061EA859216E7
:105D3000CDB305117BDE31426D2BADB12DD8393D90
:105D40000F7FC3F847A232276ECEE52750073CBC31
:105D5000C76592BFC17AE65FF388D53D6056F4C34C
:105D600016799492F556E325949CBE2CEED3B0F4AC
:105D7000FE639D9F963758E38EFC67ED163F07FC48
:105D80002ED1F74A50EB2DE5E4C4992EEA6E677FD9
:105D9000C3269A2CBC9F357C2182DE95903610DE7E
:105DA0003C8F0D311493E03684E9A3E75A18E802DA
:105DB000F242A4B674CEB0D418CE29BDB2C1F5E576
:105DC0009AE05125861D698EF28C53CDF2251E5620
:105DD000554E4A0871E15874BA11B72CA84D86E6A1
:105DE000238FDB6BFEB22E6E0AAC2F316E931CD765
:105DF0004806F85C8C8E2D9D20116B869B8CF7B924
:105E000090FB024276D4CBD63BF01E792C37D96D6D
:105E1000428BA4156F982262740DB4125DF6443D56
:105E200093B86A4511B9A3AB20B6AD43B0B4792E8F
:105E3000FE409058FEB728427C1CAFF2A778BB54B6
:105E400050F8C064302A055C69F3C1225D0F487FB9
:105E5000CE7B6C7CA75FF6E5468EB32A97E5B6DA73
:105E600073EFDEAFE668AD06A3BAC168BB78928374
:105E7000A8575E9903579C05510B83B4D827BFFDE3
:105E8000C9BF31BD1862FF4618B7BC2F60D87B610F
:105E9000AF4F303776DC6E43332D9C4405EE7114E2
:105EA000C9107260C170D3A5876E82AAFBBC6EBB9D
:105EB0003FAD63A1C8E0EA85E5FA71536A5FE9F195
:105EC000B19A8482AC7BE0F7B5C95EC4101B1D5645
:105ED0002232F64044EC169065727CBBB0981B8B66
:105EE00026EBC79DC11F94E0F4B22A947D6700A100
:105EF000924A680FA24838E8E26C5F823210FC9B3D
:105F0000A774978DA783FFA95D0AA5DE310222F24F
:105F100091CF34F7E27F26E6D5CF62919246B43630
:105F20006B65EE55E848331A1B6A6F7D0E55A52E3A
:105F3000DF250168FE1A39FE8349114DACD873E2A2
:105F400079597574F34557A6DA1327BD02DD05E6C6
:105F5000D3BF1A14FE7C97ED045172797198D6C89C
:105F60009C4C559DEEEB830F9F044FBBA831733BB8
:105F700097F470DBCF29B15503597D2AEF3E9EB5CA
:105F8000CC0B6B04FA0FF81543EEFDE4CD54F73655
:105F90000A7577CDBC0D889818FD770FB3A4C1DBC7
:105FA0000B317609F0BE209A739B4AB65977B15AE5
:105FB0007A47CBEA34969C42A9CF7B5C33220166B8
:105FC00011EDB58A89EA6BBE8134760CBD95D8DDBA
:105FD0008B4620CE9B3F85AC39C67BF71F48028F8E
:105FE000882CA6FDFB237DF8641A7AC835154A264D
:105FF0006EA15137942AEA3824FC88737EA75B0A85
:00000001FF
